:020000000F28C7
:10000800FF0003088312B9000408BA000A08BB00FD
:100018007E08BC00342D1F21FC001E21FB001D2181
:10002800FA00FD011728703083168F04BA2464255E
:100038002108A1002008A00028232008A0002108EA
:0E004800A100A201A301CE22C83056251B281C
:10020000FE00FE1F082983137E18831700080800CC
:100210000408FE0001308A007E0882070034403462
:1002200057342234063415340C3408345634003430
:100230000434FF340234013404347F347F347F3497
:10024000B200B10803193229320884000008B30053
:10025000840A0008B400840A0008B500340433049A
:10026000031D46293208840000308001840A800181
:10027000840A80010800B10A32088400840A840AD2
:100280000310800C8403800C8403800CB301B40140
:10029000FE30B500320884000008B600840A000869
:1002A000B700840A0008B8003608B3053708B4055B
:1002B0003808B50535083404330403197A293B2975
:1002C000B10A3208840001308007840A0030031824
:1002D000013E031D8007840A00300318013E800799
:1002E00032088400840A840A0310800C8403800C82
:1002F0008403800CB301B401FF30B50032088400E0
:100300000008B600840A0008B700840A0008B80094
:100310003608B3053708B4053808B5053508340480
:10032000330403199D296029B103320884000310A6
:10033000800D840A800D840A800D32088400000834
:10034000B300840A0008B400840A0008B500B41F92
:1003500094293118B22932088400840A7F3080053C
:10036000840AFF300310B10C3108B300B401B501A9
:10037000B500B401B3013208840033088004840A54
:1003800034088004840A3508800408002F30B10046
:1003900025300B24AD00AF08031DD5292808A50082
:1003A0002908A6002A08A70008002E30B10028302E
:1003B0000B24AB00AE080319612A0630AC002E08EE
:1003C0002F020318082A2E08B0002F08B002193097
:1003D0003002031CF429A501A601A7012E08AF00D5
:1003E0002B08AD002D2A0310A80DA90DAA0DAE03F0
:1003F0002E082F060319FE29AC0BF3292F082E0611
:1004000003192D2A0310A70CA60CA50CAF0AFE2970
:100410002F082E0603192D2A2F08B0002E08B0022F
:1004200019303002031C192AA801A901AA012D2A9A
:100430000310A50DA60DA70DAF032E082F06031957
:10044000232AAC0B182A2F082E0603192D2A031075
:10045000AA0CA90CA80CAE0A232AAD080319392A44
:10046000FF30A506A606A706A50A0319A60A0319C2
:10047000A70AAB080319452AFF30A806A906AA0651
:10048000A80A0319A90A0319AA0AAD012808A50791
:10049000290803110318290A031DA6072A080311B6
:1004A00003182A0A031DA707A71F612AFF30A50604
:1004B000A606A706A50A0319A60A0319A70AAD01ED
:1004C000AD0A2F08B10025302021AD08031908001E
:1004D0008030A7060800AE01AF01B0012C30B1009A
:1004E00025300B24AB002D30B10028300B24AB0697
:1004F000AD08031DAC08031D842A2E08A5002F0893
:10050000A6003008A70008002D087B3EAC07073086
:10051000AD00251C992A2808AE07290803110318E5
:10052000290A031DAF072A08031103182A0A031D0D
:10053000B0070310A70CA60CA50C0310A80DA90D5D
:10054000AA0DAD0B892A0930AD00251CB52A280853
:10055000AE07290803110318290A031DAF072A084B
:10056000031103182A0A031DB0070310A70CA60CD9
:10057000A50C0310B00CAF0CAE0CAD0BA52A2C08CB
:100580008313B1002E302021AB08031DB0172E08B5
:10059000A5002F08A6003008A70008006430AC00B2
:1005A000AD01AE01AF012308AB002208AA0021086B
:1005B000A9002008A800C3232808013E0921FA0049
:1005C000403A031DE52AFA01FA036430AC00AD019C
:1005D000AE01AF012308AB002208AA002108A90040
:1005E0002008A80084242B08A7002A08A6002908B0
:1005F000A5002808A4000A30AC00AD01AE01AF018F
:100600002708AB002608AA002508A9002408A8008E
:10061000C3232808013E0921FB000A30AC00AD01CC
:10062000AE01AF012708AB002608AA002508A900E3
:100630002408A80084242B08A7002A08A60029085B
:10064000A5002808A4008313013E0921FC0008002E
:100650002108A6002008A500FC242508A5002608DE
:10066000A6002708A7008D30A8009730A9003D30CC
:10067000AA006B222508A2002608A3002708A400D0
:100680008D30A8001730A900C230AA002208A500AA
:100690002308A6002408A700C6212508A5002608CF
:1006A000A6002708A7001A252508A2002608A300EF
:1006B0002708A400A8012030A9004130AA00220880
:1006C000A5002308A6002408A7006B222508A20085
:1006D0002608A3002708A4002208A5002308A600D6
:1006E0002408A70078232608A1002508A0000800F8
:1006F0002A30B10025300B24A9002508AB002608BC
:10070000AC002708AD00AE018E30AA02AA1F9A2BBA
:100710002A08803A8F3E0318922BA501A601A70153
:10072000A80108000310AE0CAD0CAC0CAB0CAA0F6A
:10073000922BAC2B20302A02031CA92BA501A60169
:10074000A701A80108000310AB0DAC0DAD0DAE0D57
:10075000AA03AA08031DA32BA9080319BA2BAB09E6
:10076000AC09AD09AE09AB0A0319AC0A0319AD0A0D
:100770000319AE0A2E08A8002D08A7002C08A60011
:100780002B08A5000800B101B201B301B4012F0884
:100790002E042D042C040319022CB001B00A0310FE
:1007A000AF1BD82BAC0DAD0DAE0DAF0DCE2B031086
:1007B000B10DB20DB30DB40D2F082B02031DEA2BA2
:1007C0002E082A02031DEA2B2D082902031DEA2BFD
:1007D0002C082802031CFC2B2C08A8022D08031C43
:1007E0002D0FA9022E08031C2E0FAA022F08031C8E
:1007F0002F0FAB0231140310AF0CAE0CAD0CAC0CD0
:10080000B00BD72B3408AB003308AA003208A9007C
:100810003108A8000800B20084000008B400840A6F
:100820000008B500840A0008B6000F300310B60CAB
:10083000B50CB40CFF3E031D162C3408B300B700F2
:100840003108840037088000B308031D302C3208BB
:10085000840000308001840A8001840A800108003D
:10086000B30132088400840A80308004840A32088C
:1008700084000008B400840A0008B500840A000857
:10088000B600B61BB30A32088400840A840A8001C9
:1008900033080800AA1F602CAE01AF018030B00001
:1008A0002808AE0229080318AF03AF022A0803186C
:1008B000B003B0022E08A8002F08A9003008AA0033
:1008C000AD1F762CAE01AF018030B0002B08AE0218
:1008D0002C080318AF03AF022D080318B003B002B1
:1008E0002E08AB002F08AC003008AD008030AA06FF
:1008F000AD062D082A02031D08002C082902031D3D
:1009000008002B08280208002F082E042D042C04B0
:1009100003190800B001B00AAF1B942C0310AC0DF2
:10092000AD0DAE0DAF0D8B2C2F082B02031DA22C8D
:100930002E082A02031DA22C2D082902031DA22C19
:100940002C082802031CB32C2C08A8022D08031C19
:100950002D0FA9022E08031C2E0FAA022F08031C1C
:100960002F0FAB020310AF0CAE0CAD0CAC0CB00BE8
:10097000942C0800073083129900083083169100E8
:100980001130831285001030831685008312FF30EA
:100990008700831687018D3083129F0083169F1670
:1009A000013083129000CB308F00F6308E0083161A
:1009B0000C1483120C100B178B17080027308500BE
:1009C0003F30870003307D020318FD017D087A3E29
:1009D0008400000887007D080C3E0921073ABD000D
:1009E0007D087A3E840000084039BE0003103E0CAA
:1009F0003D048500FD0A080026082504031D042D7A
:100A0000A501A601A70108002508AB002608AC0037
:100A1000AD012B08A8002C08A9002D08AA008E30D3
:100A2000B100283020212808A5002908A6002A089E
:100A3000A7000800AB01AC01AD012508A8002608FD
:100A4000A9002708AA004A24031808002508A800BE
:100A50002608A9002708AA0047252808A500290874
:100A6000A6002A08A70008000C1C3C2D0C10CB3057
:100A70008F00F6308E00DE243C08FE003B088A0022
:100A80003A08840039088300FF0E7F0E0900003009
:100A90002A06031D512D00302906031D512D00305B
:100AA0002806031908008030AA060800A0000430B8
:100AB000A1007D30F0000000F00B5B2D6400A10B65
:100AC000592DA00B572D08009F149F18652D8316D4
:100AD00083121E08A10083161E088312A0000800BE
:02400E00C430BC
:00000001FF
